:020000002028B6
:08000800A1000308A2000B1D7A
:100010001C280B1162308100201C13288601240843
:100020008700201017288701230886002014A50BBD
:100030001C281E30A500A0142208830021080900F6
:1000400083160313803086000F3085000730870049
:100050000E309F00831203178D01831603178C1334
:100060000C14831203170C0883120313A800A014A6
:10007000A301A4011E30A500623081008316031382
:10008000C530810083120313A0308B00A01C85288B
:10009000A01081309F001E30A600A60B4D281F1512
:1000A0001F1950281E08A7001F10A70CA713201DFA
:1000B0005D2828082702A900642827080319632857
:1000C0002807A9006428A90007308A00270800270C
:1000D000A30006308A0027080026A40005198528F9
:1000E00027087F3C0319822803187C2820157F30BD
:1000F0002702A800B5208528201127087F3CA800EA
:10010000B52085282011A801B5202308EE3C03194D
:100110008B28A01194282408D73C03199128A011FA
:10012000A228A0152012A2282308FB3C03199A2814
:100130002012A2282408FD3C0319A0282012A2287E
:100140002016A0110718A9288511861BAF28851233
:100150004628201AAD288515AF2885114628A019F4
:10016000B32885164628851246288B132808831243
:1001700003178C008D01831603178C130C15553053
:100180008D00AA308D008C148C18C4280C11831299
:0801900003138B170B1108008B
:100C00008207FD34FD341534BB349F349F34573490
:100C1000CF346F3495349534FF34D734FD341534E4
:100C20001534BB349F3457345734CF346F34953434
:100C3000FF34FF34D734FD341534BB34BB349F3418
:100C40005734CF34CF346F349534FF34D734D7345E
:100C5000FD341534BB349F349F345734CF346F3454
:100C600095349534FF34D734FD34FD341534BB341A
:100C70009F3457345734CF346F349534FF34FF34B6
:100C8000D734FD3415341534BB349F345734CF3446
:100C9000CF346F349534FF34D734D734FD34153422
:100CA000BB34BB349F345734CF346F346F349534F6
:100CB000FF34D734FD34FD341534BB349F345734FE
:100CC0005734CF346F3495349534FF34D734FD34F2
:100CD00015341534BB349F345734CF34CF346F348C
:100CE0009534FF34FF34D734FD341534BB34BB3472
:100CF0009F345734CF346F349534FF34D734D734DE
:020D0000D734E6
:100E00008207FB34FB34FB34FB34FB34FB34FB3410
:100E1000FB34FB34FB34FB34FB34FB348A348A343C
:100E20008A348A348A348A348A348A348A348A34D2
:100E30008A348A348A34DD34DD34DD34DD34DD3423
:100E4000DD34DD34DD34DD34DD34DD34DD34DD341A
:100E5000CF34CF34CF34CF34CF34CF34CF34CF347A
:100E6000CF34CF34CF34CF34AE34AE34AE34AE34EE
:100E7000AE34AE34AE34AE34AE34AE34AE34AE3462
:100E8000AE34E734E734E734E734E734E734E734C3
:100E9000E734E734E734E734E734E734B734B734DA
:100EA000B734B734B734B734B734B734B734B734EA
:100EB000B734B734CA34CA34CA34CA34CA34CA3468
:100EC000CA34CA34CA34CA34CA34CA34CA34FF34FD
:100ED000FF34FF34FF34FF34FF34FF34FF34FF347A
:100EE000FF34FF34FF34FF34EE34EE34EE34EE34AE
:100EF000EE34EE34EE34EE34EE34EE34EE34EE34E2
:020F0000EE34CD
:02400E00010FA0
:00000001FF
